:020000020000FC
:100000008EC08CC08BC08AC064C088C087C06AC0E4
:1000100085C084C083C078C081C018C07FC07EC046
:100020007DC07CC06AC085990FC0AA20D9F0202E5F
:1000300009E0A01630F00DE0A01618F40894111C89
:10004000BB24AA24022D0EC0A3940CC00FB6B394F7
:1000500052F341F4110CAA24969904C0202E08E30F
:10006000B02E022D0FBE1895992431016418750821
:1000700058F43201621873086818790808F4089572
:1000800012012818390808956818790808F40895A5
:100090001201280C391C0895DF93CF9308BBC0E6EA
:1000A000D0E00770000FC00F28803980E1990CC0A4
:1000B000210128883988CEBBE09A8DB2882012F0C1
:1000C00009F0D2DF288239823BBC2ABCCF91DF9174
:1000D00008950FB60F9308B3077F0395DDDF0F91E7
:1000E0000FBE18950FB62CB02D92AF71A0680FBE41
:1000F000189524B2239424BA08950FB69899F9DF7D
:10010000C49B849A0FBE18950FB60F936F937F937D
:1001100006D37F916F910F910FBE189518950FED33
:100120000DBF77D061E189D0672F6770671361E0F9
:100130007727660FF7E0E2E9E60FF71F05911591C3
:1001400012B909B90EE003B908E90AB902E00BB91E
:10015000A0E8B0E0CD016D01F7E0E2EA03C05D9BED
:10016000FECF0CB905910023D1F70DE706BF02E0E1
:1001700000BF02E003BF1CE005E315BD04BD00EFB6
:100180008BDF01E409BF02E80FBD0AE10EBDA895AF
:10019000002704BF01B5086101BD05E401BD8CD293
:1001A000B9D200E20BBF0FE107BB00E402BB00E5E0
:1001B00001BB65E142D070FD949A7894A81386D073
:1001C000AC11B8D2989903D0BED2C9D2F7CF62E1B0
:1001D00034D064B367130895C49B07C094990895FD
:1001E000F89417D07894C498949A002704BB60E3DD
:1001F00024D077FD08958B0164E11FD0572FB801FB
:1002000001C01BD05D9BFECF7CB963955A95C9F7A1
:1002100008956627C0E6D0E010D0072F63950DD073
:10022000172F639517FF02C003E517E0088B198BA2
:1002300009931993603181F70895E199FECF0F93E7
:100240000FB7F8946EBBE09A7DB30FBF0F9108957E
:10025000B69B08950F93072FF0DF071731F0F8943E
:100260006EBB0DBBE29AE19A78940F9108952991A3
:10027000CF71C068089509917027CF71C068089543
:100280000991CF71C0680F7406FD0753F991CF71C2
:10029000C068FF74F6FDF75302950F2B0895EBDF4E
:1002A0000F7406FD0753F9917F27CF71C068FF7463
:1002B000F6FDF75302950F2B0895DDDF0A3209F0A2
:1002C0000895DEDF0F3F09F007170895EC017C0168
:1002D0006A2F681B08F4605E633008F40895099182
:1002E000CF71C068CE010F3F51F51991CF71C06831
:1002F0001F3F09F40895BBDF2F3F09F40895CE0195
:1003000060E19BDF77FD7727770F770F770F68EF37
:10031000612367130895177031E028503040A90118
:10032000220F331F220F331F240F351FC0E7D0E0E9
:10033000110FC10FF89428833983789408950038F9
:1003400069F41991CF71C068212F27702113089586
:100350003327F2E0E4EBE20FF31F0994043249F48F
:100360007AE219917127CF71C0681F7D1534C9F0E9
:10037000089515B301130895562F63E15EDF5717F3
:1003800010F4C7010895572F60E206C01991CF718C
:10039000C06853DF1713089563955A95B9F7CE01D6
:1003A000BEC1653010F4C701089587DF19F00C3223
:1003B00011F00895B4C173DF0F3FD1F46E3010F423
:1003C000C701089558DF0C3209F0089568DF0F3F28
:1003D00009F40895102F4FDF0C3209F008955FDF04
:1003E0000F3F09F40895202F68DF09F0089587CFA3
:1003F0000038B9F46C3010F4C70108953CDF0C32BA
:1004000009F008954CDF202F27702013089533DF63
:100410000C3209F008953327F2E0E2E1E20FF31F16
:100420000994089507C012C03BC048C055C060C0C1
:1004300077C08EC06E3010F4C701089530DF07FD1D
:100440000895202F3ADF09F0089599C0643110F41F
:10045000C701089524DF033020F0673110F4C7018D
:100460000895202F08DF0C3209F0089518DF07FDEA
:100470000895302F00DF0C3209F0089510DF07FDDA
:100480000895402F233040F0F6DE0C3209F0089535
:1004900006DF07FD0895502F10DF09F0089596C07C
:1004A0006E3010F4C7010895FADE202F2F7020134C
:1004B000089503DF09F00895722FC7C06E3010F45D
:1004C000C7010895ECDE202F277020130895F5DE74
:1004D00009F00895722FC1C06E3010F4C70108955D
:1004E000DEDE07FD0895202FE8DE09F00895BBC089
:1004F00055276B50E0EAF0E029917227CF71C06870
:1005000027FD089521932A3239F053955B3019F075
:100510006A9591F7C7010895D4DE09F00895C6C021
:1005200055276B50E0EAF0E029917227CF71C0683F
:1005300027FD089521932A3239F053955B3019F045
:100540006A9591F7C7010895BCDE09F00895C9C006
:100550006E3010F4C7010895A2DE07FD0895202F24
:10056000ACDE09F00895D2C007C012C069C070C0E7
:1005700077C08BC0A5C0C7C07ADE27FD0895CE0125
:100580007CE502D0622F59DE5D9BFECF7CB90895D9
:10059000653010F4C70108956ADE27FD0895233001
:1005A00020F0663010F4C70108953991CF71C0680A
:1005B00037FD08954991CF71C06847FD08952330F4
:1005C00028F05991CF71C06857FD0895CE0160E1C0
:1005D00034DE77FD7727770F770F770F68EF632388
:1005E000671308953770213029F0243041F0253009
:1005F00001F1089560E6330F630F742F29CE550F74
:100600004695579518EB0BE05117400718F041F04D
:10061000A80106C01EEE02E05117400708F4A80129
:10062000C0E7D0E0330FC30FF89458834983789420
:100630000895E5DF632F752F0BDE6395742F08CEC9
:1006400016DE722F7F7072130895CE0160E100CE26
:100650000EDE722F777072130895CE0161E1F8CD2E
:1006600006DE27FD0895CE0162E1722FF1DD989834
:100670009498C49A62E1E1DD7F77739577FD0895E0
:10068000989AA895002704BB089555276250E0EA80
:10069000F0E0EDDD27FD08952193222339F05395F5
:1006A0005A3021F06A95A9F7C7010895CE0163E198
:1006B000752FCEDD60E21AD060E2BFDD75BBD7CF0B
:1006C00055276250E0EAF0E0D2DD27FD089521933E
:1006D000222339F053955A3021F06A95A9F7C701C2
:1006E0000895CE0164E1752FB3DD60E37FEFB0DDE7
:1006F000552309F40895E0EAF0E07191A9DD6395CE
:100700005A95D9F70895B3DD27FD0895CE0165E127
:10071000722F9EDD65E191DD707270BD089565E117
:100720008CDD74FF02C0B79B0895C499A0CF70FF01
:100730009ECF08955D9B0895E6010991CF71C06831
:100740000CB96E01089565E178DD74FF0895C49BCE
:1007500003C0B79B43CD0895989BE1CF0895012D29
:100760000F7165E16ADDC49902C070FD06C00F31EA
:1007700021F4969870FDA8950895969908951127EB
:10078000F7E0E0EDE00FF11F049100FDF3CF969A42
:10079000089508028100560040002A00200015003C
:1007A0000A004D696C6C73776F6F6420456E6769E2
:1007B0006E656572696E67204661696C7361666516
:1007C000204465766963652056312E32340D0A0067
:1007D00000000000000000FF000000FF00FFFFFF1E
:1007E000000000FF00FFFFFF00FFFFFFFFFFFFFF14
:00000001FF
